:100000000C94AE010C94E6010C94E6010C94E6010C
:100010000C94E6010C94E6010C94E6010C94E601C4
:100020000C94E6010C94E6010C941D1A0C94EF1A42
:100030000C942F150C94E6010C94E6010C94E60147
:100040000C94E6010C94E6010C94E6010C94E60194
:100050000C94E6010C94B7150C94E6010C94E6019F
:100060000C94E6010C94E6010C94E6010C94E60174
:100070000C94E6010C94E6010C94E6010C94E60164
:100080000C94E6010C94E6010C94E6010C94E60154
:100090000C94E6010C94E6010C94E6010C94E60144
:1000A0000C94E6010C94E6010C94E601130413048D
:1000B0003F043F04A704D205D205D205C5045E055E
:1000C0006F056F055C1B831B7B1C831B7B1CCF1B7D
:1000D000F21B7B1C491C581C290000003A003B0005
:1000E0003C003D003E003F00400041004200430014
:1000F0004400450046004700480035001E001F0030
:1001000020002100220023002400250026002700D3
:100110002D002E002A0049004A004B002B0014003D
:100120001A000800150017001C0018000C0012002F
:1001300013002F00300031004C004D004E003900FC
:1001400004001600070009000A000B000D000E0055
:100150000F00330034000000280000000000000001
:10016000E10000001D001B00060019000500110041
:100170001000360037003800E50000000000520093
:100180000000E000E300E2000000000000002C009E
:10019000000000000000E6000151E700E40050000C
:1001A00051004F00010000000100010001000100AA
:1001B0000100010001000100010001000100010037
:1001C000C05CBE5CBF5C01000100010001000100D9
:1001D0000100010001000100010001000100010017
:1001E000010001000100A90001000100010001005F
:1001F000005C01000100010001000100010001009C
:1002000001000100AE00AB00AA00010001000100E6
:1002100001000100010001000100010001000100D6
:1002200001000000010000000000000001000000CB
:1002300001000100010001000100010001000100B6
:1002400001000100010000000000010000000100A9
:10025000010001000000000000000100000000009B
:100260000000010001000100010001000100010087
:100270001003650070006F006300680038003000F4
:1002800000001403630061007200790077006F00C2
:1002900072006B00730000000403090409023B00B4
:1002A000020100A0FA090400000103010100092174
:1002B0001101000122400007058103080001090423
:1002C0000100010300000009211101000122320098
:1002D00007058203200001120100020000000863EC
:1002E00064000001000102000105010980A10185EF
:1002F0000319012AB700150126B700950175108171
:1003000000C0050C0901A101850419012AA00215EC
:100310000126A002950175108100C005010906A102
:1003200001050719E029E7150025019508750181E8
:10033000029501750881010507190029FF1500269E
:10034000FF00950675088100050819012905950526
:1003500075019102950175039101C00011241FBE22
:10036000CFEFDAE0DEBFCDBF04B603FE18C0809148
:10037000A3029091A402A091A502B091A602873099
:10038000904BA740B04B59F41092A3021092A402D4
:100390001092A5021092A602E0E0F8E3099511E0A0
:1003A000A0E0B1E0ECE0FAE302C005900D92AA38BB
:1003B000B107D9F722E0AAE8B1E001C01D92A33A43
:1003C000B207E1F70E940D120C94041D0C9400007A
:1003D00081E0089581E008950C94EA0108950C9459
:1003E000EE011F93CF93DF9300D000D01F92CDB7C3
:1003F000DEB749835A836B8330918D0189819A815D
:10040000311114C0662359F0222349F00E940B08D1
:10041000182F682F89819A810E94B40703C00E9417
:10042000DF07182F69817A81812F04C00E940B0891
:1004300069817A810F900F900F900F900F90DF914C
:10044000CF911F910C94570FFC01262F40815181B1
:100450006281738184810C94F10181E00895CF93CE
:10046000DF93EC0160E00E942402BE01DF91CF9196
:100470000C94EF010C94A0100C949C1008950E9411
:100480005E060E943E022FEF84E39CE021508040F4
:100490009040E1F700C000000C94DD150F931F930E
:1004A000CF93DF938C0161E00E942402EC01B8013C
:1004B0000E94EC018823F1F1B801CE010E940614DC
:1004C0008823C1F1B801CE010E941A12882391F14C
:1004D000B801CE010E946213882361F1F801828184
:1004E000882309F1CB358DE5D807C1F050F4C1154B
:1004F000FCE5DF0781F0CF3DDC45A9F40E94420D09
:1005000019C0CC35EDE5DE0761F0CD35DD4559F498
:100510000E94850C08C00E943F020CC00E948E0CF5
:1005200002C00E94910CC801DF91CF911F910F91E1
:100530000C94E80180E0DF91CF911F910F91089515
:100540000E940F150C94CE020E94D1020C94151536
:1005500008950C94A80281E00895CF93C82F0E94BB
:10056000AB02882359F0C095C1FF02C0769A01C042
:100570007698C2FF02C02F9A01C02F98CF9108959C
:100580006E9A769A279A2F9A0895CF93C82F0E9431
:10059000A9028C2F0E94AD02CF91089580E00C94A7
:1005A000C5020E9462140C94C5020E9462149091CC
:1005B0008C01891721F080938C010C94C502089559
:1005C000CF93DF93CDB7DEB72B970FB6F894DEBF8E
:1005D0000FBECDBF4F83588769877A878B8761119C
:1005E0000E94D10B9E012F5F3F4F86E0F9011192CF
:1005F0008A95E9F785E0FE013796D90101900D92C1
:100600008A95E1F789819A814C815D81452B31F092
:100610009F3F31F491E08F3F19F403C091E001C096
:1006200090E090FF09C049815A816B817C818D8166
:100630009E810E94F20A05C0C9010E942D0281110B
:10064000F2CF2B960FB6F894DEBF0FBECDBFDF9171
:10065000CF910895FC01808191810E944D080895F9
:10066000CF93882309F448C0C82F8CEF8C0F813AB0
:10067000D0F46C2F80910201909103010E94B1147B
:10068000882349F06C2F80910201909103010E9410
:10069000E9140E94F30B6C2F8091020190910301E9
:1006A0000E94E7140CC080E28C0F883058F4C770A9
:1006B00081E001C0880FCA95EAF70E94B40BCF9180
:1006C0000C94F30BEBE5EC0FE33040F4F0E0E15C6D
:1006D000FE4F808190E0CF910C947914C85AC731B5
:1006E00058F4EC2FF0E0EE0FFF1FEF5EFE4F80811D
:1006F0009181CF910C948F14CF910895882349F163
:10070000682F8CEF860F813A38F480910201909126
:1007100003010E94E9140CC080E2860F883050F477
:10072000677081E001C0880F6A95EAF70E94BA0BF2
:100730000C94F30B8BE5860F833020F480E090E07F
:100740000C947914685A673120F480E090E00C949E
:100750008F1408951F93CF93DF93182FEB010E94FE
:100760003003209741F08FE99FE00197F1F700C037
:1007700000002197F6CF812FDF91CF911F910C942C
:100780007E03893319F060E070E002C060E570E03C
:100790000C94AA03882321F00E94B40B0C94F30B51
:1007A0000895882321F00E94BA0B0C94F30B08954E
:1007B000CF92DF92EF92FF920F931F93CF93DF932D
:1007C0007C01D62FC72FFC011281058102950F7085
:1007D0000E94AA0B8823B9F01123A9F08C2F807FE7
:1007E000803421F080E28D0F883068F080916102C2
:1007F00082FD09C082E00E94530C0E94AA0B91E086
:10080000D82ED92601C0D12CCC2EC2948FE0C8227C
:100810008C2D90E08C30910508F0C4C1FC01EA5A9F
:10082000FF4F0C94AF1C8C2F807FCF70882311F06A
:10083000C295C07F112399F0CC2309F49FC180E2B7
:100840008D0F883010F0D11104C08C2F0E94B40B92
:1008500003C08C2F0E94C40B0E94F30B8FC18D2FFD
:100860000E947E03CC2309F49DC180E28D0F883065
:1008700038F1DD2329F18C2F0E94CA0B24C08C2F64
:10088000807FCF70803211F0C295C07FDD2319F0D8
:10089000D130A1F13DC08091610282FF17C01123C8
:1008A00049F0CC2329F08C2F0E94B40B0E94F30B4B
:1008B00080E065C180E00E947E03CC2309F472C110
:1008C0008C2F0E94BA0B0E94F30B6CC1112371F0A4
:1008D000002341F0013031F40E94D40B8C2B0E9494
:1008E000DC0B60C10E94D40B8C2B1DC0002319F0BF
:1008F000013009F457C10E94E90B25C0112321F0F2
:10090000063008F04FC10EC0053008F04BC11BC0C7
:10091000112361F0002331F0F701858180FF2EC1A2
:100920008F7085838C2F0E94CA033CC1002359F02D
:10093000D93309F034C1FFEF07EE13E0F150004066
:100940001040E1F72AC18C2F0E94D1032BC18C2FBC
:1009500086958695837019F0813061F023C111234B
:1009600021F08D2F9C2F937002C080E090E00E94B8
:10097000791420C1112321F08D2F9C2F937002C078
:1009800080E090E00E948F1415C18C2F837009F0D5
:1009900047C011110BC12D2F229526952770220FCC
:1009A000220F6D2F6F70862F90E0A0E0B0E0022E36
:1009B00004C0880F991FAA1FBB1F0A94D2F7D4FF47
:1009C00010C04FE050E060E070E004C0440F551FDD
:1009D000661F771F2A95D2F74095509560957095C0
:1009E00003C040E050E0BA01C695C695C3708A01C5
:1009F0009B01082B192B2A2B3B2BC901B801C230B4
:100A000049F058F4C13019F00E94CA06CFC00E94C4
:100A1000B806CCC00E94DC06C9C00E94B606C6C09B
:100A2000112319F08C2F817001C08695882309F459
:100A3000BDC02D2F229526952770220F220F6D2FD6
:100A40006F70862F90E0A0E0B0E0022E04C0880F07
:100A5000991FAA1FBB1F0A94D2F7D4FF10C04FE002
:100A600050E060E070E004C0440F551F661F771F20
:100A70002A95D2F7409550956095709503C040E057
:100A800050E0BA01C695C695C3708A019B01082B38
:100A9000192B2A2B3B2BC901B801C23049F058F45D
:100AA000C13019F00E948F0781C00E947D077EC06F
:100AB0000E94A1077BC00E94F00678C0CF7011236E
:100AC00039F08C2F0E9416078D2F0E94CA036EC02A
:100AD0008D2F0E94D1038C2F0E94370767C0D23F11
:100AE00021F128F4D03F41F0D13FC1F043C0D33FC2
:100AF00019F1D43F79F03EC0112341F0053008F0E0
:100B000051C08C2F8F710E945C074CC0063008F0DA
:100B100049C0F7CF8091610282FF18C0112339F0DC
:100B20008C2F8F710E9416073DC01123C9F38C2FA3
:100B30008F710E94370736C0112329F08C2F8F71D7
:100B40000E9401072FC00E94FC062CC0112349F00F
:100B5000CF718C2F0E94160763E08C2F0E94380CF7
:100B600021C081E00E94530C0230E0F082E00E943C
:100B7000530C18C0112331F0002391F28D2F0E94E5
:100B8000300310C0002399F2D93349F41FEF27EE48
:100B900033E0115020403040E1F700C000008D2FBD
:100BA0000E947E0388EF8C0D843020F40E94621432
:100BB0000E94C502DD20C9F00E94A60B80FD15C071
:100BC000F70112820E94A00B0E941607C7010E9423
:100BD00016060E94A00BDF91CF911F910F91FF90FD
:100BE000EF90DF90CF900C943707DF91CF911F915A
:100BF0000F91FF90EF90DF90CF9008950F931F9388
:100C0000CF93DF93EC01688179818A810E94580833
:100C10008C010E94B3070E94A406B801CE010E9475
:100C2000D803DF91CF911F910F910895CF93DF9358
:100C3000EC01988189812B813C81232B31F08F3FFE
:100C400031F481E09F3F19F403C081E001C080E0EE
:100C500080FD1DC0CE010E944E02811110C00E9475
:100C6000AA0B8823A1F08A81882389F080916102F0
:100C700082FD0DC082E0DF91CF910C94530CCE0128
:100C80000E94FE05CE01DF91CF910C942F02DF91DF
:100C9000CF91089580E090E00E94791480E090E088
:100CA0000E948F140E94D10B0C94F30B80910201CF
:100CB000909103010E94EB140C944A060E94C10B10
:100CC0000C94560692959F70963079F010F49250DD
:100CD00001C09A50923068F4803F69F018F4883E61
:100CE00040F409C0843F29F406C0883E20F0813FCB
:100CF00011F080E0089581E00895FC0180819181E8
:100D00000E944D080E9462060895CF93DF9300D0A1
:100D100000D01F92CDB7DEB70F900F900F900F90BD
:100D20000F90DF91CF910895CF93DF9300D000D043
:100D300000D0CDB7DEB726960FB6F894DEBF0FBE53
:100D4000CDBFDF91CF910895089508950C94A50625
:100D50000C94A6060E94A8066093D3017093D40158
:100D60008093D5019093D6010C944A060C94AA0660
:100D70000F931F930091D3011091D4012091D501BD
:100D80003091D601602B712B822B932B1F910F91E9
:100D90000C94AA060F931F930091D3011091D401D4
:100DA0002091D5013091D6016023712382239323B2
:100DB0001F910F910C94AA060F931F930091D301DA
:100DC0001091D4012091D5013091D601602771276F
:100DD000822793271F910F910C94AA060C94A506C5
:100DE0000E94EE066093CF017093D0018093D101F1
:100DF0009093D2010C944A0660E070E0CB010C9411
:100E0000F0060F931F9341E050E060E070E08A012C
:100E10009B0104C0000F111F221F331F8A95D2F7B8
:100E2000C901B8011F910F910C94F0060F931F9305
:100E300041E050E060E070E004C0440F551F661FC1
:100E4000771F8A95D2F78091CF019091D001A09120
:100E5000D101B091D2018A019B01082B192B2A2BB9
:100E60003B2BC901B8011F910F910C94F0060F9311
:100E70001F9341E050E060E070E004C0440F551F54
:100E8000661F771F8A95D2F74095509560957095AB
:100E90008091CF019091D001A091D101B091D20168
:100EA0008A019B01082319232A233B23C901B80186
:100EB0001F910F910C94F0060F931F9341E050E0A7
:100EC00060E070E004C0440F551F661F771F8A95CD
:100ED000D2F78091CF019091D001A091D101B09132
:100EE000D2018A019B01082719272A273B27C9011C
:100EF000B8011F910F910C94F0060F931F9300916E
:100F0000CF011091D0012091D1013091D201602BFD
:100F1000712B822B932B1F910F910C94F0060F9342
:100F20001F930091CF011091D0012091D1013091F8
:100F3000D20160237123822393231F910F910C947C
:100F4000F0060F931F930091CF011091D0012091D3
:100F5000D1013091D20160277127822793271F91F9
:100F60000F910C94F006089521E1929F800D1124B9
:100F7000E82FE695E695E695877051E001C0550F9C
:100F80008A95EAF785E0E89FF0011124E257FE4FC9
:100F900020E030E070E04081CB01022E02C0969547
:100FA00087950A94E2F781708195842785238427A9
:100FB00081932F5F3F4F2530310569F7089521E177
:100FC000929F800D1124682F669566956695982FDF
:100FD000977085E0689FB001112440E050E080E008
:100FE000FB01E40FF51FE257FE4F208130E0092E90
:100FF00002C0369527950A94E2F721703327042E14
:1010000001C0220F0A94EAF7822B4F5F5F4F4530F1
:10101000510531F70895BF92CF92DF92EF92FF9280
:101020000F931F93CF93DF938C01C090CF01D0908B
:10103000D001E090D101F090D2018091D301909144
:10104000D401A091D501B091D601C82AD92AEA2AA3
:10105000FB2ACFE1D0E0D701C6010C2E04C0B69523
:10106000A795979587950A94D2F780FD04C021979C
:1010700090F7B12C07C0BC2EB8018C2F0E946A0FCC
:101080000197A9F38B2DDF91CF911F910F91FF90C5
:10109000EF90DF90CF90BF900895CF93DF93EC0156
:1010A0000E940B08BE010E946A0FDF91CF91089544
:1010B0001F93CF93DF93EB0190918D01992321F042
:1010C000CB010E944D0813C0882349F0CB010E9438
:1010D0000B08182F682FCE010E94B40704C0CB0163
:1010E0000E94DF07182FBE01812F0E946A0FDF9137
:1010F000CF911F9108951F93CF93DF93C091D70194
:1011000016E08091D801C81799F0D0E01C9FF0013B
:101110001D9FF00D1124E752FE4F408151816281E5
:101120007381848195810E9494062196C770E9CFCE
:10113000DF91CF911F9108954091090250910A02C9
:1011400060910B0270910C0280910D0290910E0241
:101150000C949406EF92FF920F931F93CF93DF931B
:1011600080910E0282958F7009F065C080910B020C
:10117000882309F460C08091D701F090D8011091C4
:10118000090200910A0260910C0270910D0291E037
:101190001F3F09F090E0C0910001D0910101292F7B
:1011A00096E0E92E8F1509F446C06115710521F00E
:1011B0000F3F21F030E003C031E001C0322F90E05A
:1011C00030FD36C0E89EF001E99EF00D1124DF01EC
:1011D000A752BE4F11963C911197301329C03C91F4
:1011E000311326C012963C911297311121C01396EB
:1011F0004D915C911497461B570B4C175D07C0F43B
:1012000080910E028F70806180930E02E252FE4F39
:1012100080818F708061808389E092E00E94160651
:10122000DF91CF911F910F91FF90EF900C947B086D
:1012300001968770B7CFDF91CF911F910F91FF90EB
:10124000EF9008959F92AF92BF92CF92DF92EF926C
:10125000FF920F931F93CF93DF93CDB7DEB76197C4
:101260000FB6F894DEBF0FBECDBF8C0185E0F8014C
:10127000DE011D9601900D928A95E1F7D801129634
:10128000EC9090910902E0910A0220910C023091B9
:101290000D022115310531F0EF3F31F481E09F3F20
:1012A00019F403C081E001C080E0B82FB1709B2E1B
:1012B00080FD47C1D8014C9111965C91119713960E
:1012C000AD90BC90149789E0C82E82E0D82EF090A3
:1012D0000B02B501621B730B2091000130910101DB
:1012E000FF2009F4D9C080910E026217730708F03D
:1012F00095C0282F207F09F052C05E1313C04913F8
:1013000011C0FE2CE1100EC08F70806180930E0220
:101310000E949C08C6010E94160680910E02F801E8
:1013200085834DC1AB2831F05F3F31F481E04F3F01
:1013300019F403C081E001C080E080FD03C081E0BA
:101340008E2502C080E090E0F82FF170FF2E80FF24
:101350001CC08091D7012091D80136E0821709F492
:101360000BC190E0389FF001399FF00D1124E75236
:10137000FE4F6181561306C06081461303C062812F
:10138000E61203C001968770E9CFFE2CEE2009F427
:1013900016C180910E02816080930E0254C05E13CC
:1013A00006C0491304C0E11002C0F80199C0C80189
:1013B0000E947D06882361F1EE2051F120910E02FA
:1013C000822F82958F7090E0029774F080910902CD
:1013D00090910A0298878F831986BB86AA862C87EC
:1013E000CE0107960E94160686E0F801A9E0B2E059
:1013F00001900D928A95E1F70E94AA080E949C082C
:101400000AC05E1711F1C8010E947D0681112CC02F
:10141000C8010E941606FF24F394D1C0282F207F14
:1014200081F77A2DB98AA88A6E2D89890E9485064E
:1014300089E092E00E94160686E0D6011D928A9508
:10144000E9F70E949C08F12CBAC04913DCCFE110E7
:10145000DACFF8018583C8010E94160686E0D6011E
:101460001D928A95E9F7ABC0EE2091F220910E0211
:10147000822F82958F7090E002970CF4B5CF809107
:10148000090290910A029A8389831B82BD82AC82F1
:101490002E83CE010196A6CF6217730708F044C0D1
:1014A000FE2CEE2009F4B4CF5E1330C049132EC0D9
:1014B00020910E0220FD21C0822F82958F70482F2F
:1014C00050E041155105C9F0F80125834F30510511
:1014D00041F08F5F982F9295907F822F8F70892B8C
:1014E0008583C8010E94160686E0F801A9E0B2E0F3
:1014F00001900D928A95E1F73CC086E0F801A9E0E1
:10150000B2E001900D928A95E1F759C0C8010E949E
:101510007D06811169CF80910E02816080930E0259
:10152000C8010E9416064BC07A2DB98AA88A6E2D72
:1015300089890E94850686E0D6011D928A95E9F781
:1015400018C0EE2009F464CFC8010E947D06F82E71
:10155000882309F45DCF86E0F801A9E0B2E00190AC
:101560000D928A95E1F789E092E00E942A030E9499
:10157000AA080E949C0823C04D875E878D859E85A2
:101580000E944D08292F22952F70223028F49F7039
:1015900039F0811105C00BC0243028F49F7049F444
:1015A000805E883020F0C8010E9416069F2CF92C1E
:1015B00006C0D80115969C91907F91F7F8CF8F2D9A
:1015C00061960FB6F894DEBF0FBECDBFDF91CF910D
:1015D0001F910F91FF90EF90DF90CF90BF90AF9051
:1015E0009F9008951F93CF93DF93CDB7DEB72C97CD
:1015F0000FB6F894DEBF0FBECDBF4F835887698703
:101600007A878B879C87CE0107960E9422098823C0
:10161000D1F09F8188852A853B85232B31F08F3F30
:1016200031F481E09F3F19F403C081E001C080E004
:1016300080FD47C04F81588569857A858B859C855B
:101640000E9494063EC086E0FE013796DE011196A8
:1016500001900D928A95E1F7FF81E8856A857B8587
:101660006115710531F0EF3F31F481E0FF3F19F46E
:1016700003C081E001C080E080FD23C02091D8013B
:1016800030E0C9010196877099274091D70150E059
:1016900084179507F1F1F983EA837D836C8396E0E3
:1016A000929FD001939FB00D1124A752BE4FFE010F
:1016B000319601900D929A95E1F78093D8010E949E
:1016C0007B0816E08091D7019091D801891771F1BC
:1016D000189FC001112487529E4F0E94220988231F
:1016E00029F1E091D7011E9FF0011124E752FE4F2E
:1016F0004081518162817381848195810E94940629
:101700008091D70190E00196877099278093D70147
:10171000D9CF0E945E061092D8011092D701E9E05D
:10172000F2E086E0DF011D928A95E9F72C960FB66C
:10173000F894DEBF0FBECDBFDF91CF911F9108950A
:10174000809117028595859585950895809117025A
:101750008770089590911702977081E009F480E0F6
:10176000089580912202089590912202892B8093FE
:10177000220208958095909122028923809322026B
:10178000089510922202089590912102892B80934E
:10179000210208958095909121028923809321024E
:1017A00008951092210208958091180208950895D5
:1017B0000C94D70B0C94D80B9091610292FD08C049
:1017C00090911802981721F0809318020C94DA0B6C
:1017D000089580911802882329F01092180280E061
:1017E0000C94DA0B0895CF93DF93E0910201F0910E
:1017F0000301809122028083E0910201F0910301B4
:10180000908180912102892B808380911802882306
:1018100081F0E0910201F09103019081892B808396
:1018200080910201909103010E94A51481110E94F0
:10183000E90BC0910201D091030148E050E06FE054
:1018400072E0CE010E94B51C892B69F088E0FE0190
:10185000AFE0B2E001900D928A95E1F7CE01DF9101
:10186000CF910C946E14DF91CF9108950C94D70B07
:101870009091610292FD10C098E0899F900111241F
:10188000262B209317020E94160780911702859538
:10189000859585950C94360C0C94160710921702BA
:1018A00080E00C94360C209117028095822380935F
:1018B0001702982F977099F430E0482F082E000CEB
:1018C000550B2417350759F09091610292FD07C01E
:1018D0008595859585950E9437070C944E0C089543
:1018E0009091610292FB222720F9281769F080FB72
:1018F00092F99093610280916002909161020E943E
:10190000BE0C82E00C94530C08958091610282FB1E
:10191000882780F991E089270C94700C81E00C9461
:10192000700C80E00C94700C6FEF7FEF80E090E023
:101930000C94EE1C80E090E00E94CA1C21E0893EDD
:101940009E4F09F020E0822F089582E090E00C94F1
:10195000C21C83E090E00C94C21CCF9384E090E022
:101960000E94C21CC82F82E290E00E94C21C2C2F51
:1019700030E0A901582BCA01CF910895CF93C92F08
:10198000682F84E090E00E94D01C6C2F82E290E0EF
:10199000CF910C94D01CAB01BC018FE090E00C9473
:1019A000E21CAB01BC0183E190E00C94E21C60E01E
:1019B00070E0CB010C94D10C60E070E0CB010E9490
:1019C000CB0C0C94D70C69EE7EEF80E090E00E9487
:1019D000EE1C60E082E090E00E94D01C60E083E0BA
:1019E00090E00E94D01C1092D3011092D40110926A
:1019F000D5011092D60160E084E090E00E94D01CF6
:101A000060E082E290E00E94D01C60E085E090E01F
:101A10000E94D01C60E086E090E00E94D01C6FEF36
:101A200087E090E00E94D01C40E050E0BA0188E0DE
:101A300090E00E94E21C60E08DE090E00E94D01CEB
:101A400040E050E0BA0188E190E00E94E21C60E0D2
:101A500087E190E00E94D01C40E050E0BA018CE1A8
:101A600090E00E94E21C60E070E080E290E00E9462
:101A7000EE1C40E050E0BA0188E190E00E94E21CD8
:101A80000C94DC0C0C94E30C682F8EE090E00C942A
:101A9000D01C0E949C1560933F027093400280937B
:101AA00041029093420260933B0270933C02809308
:101AB0003D0290933E02089585B7806885BF85B743
:101AC000806885BF089581E008950C94630D0895A2
:101AD0000C94670D0C94670D0C946A0D0C94670DB3
:101AE0000C946E0D0C94670D0E945C0D86E490E1E1
:101AF0000E9458140E94720D0C94700D0E94680D83
:101B00000C94670D0E9460100C94C0020E9487150F
:101B10000E9464110E94820D0C946C0D2F923F92D2
:101B20004F925F926F927F928F929F92AF92BF92ED
:101B3000CF92DF92EF92FF920F931F93CF93DF9399
:101B4000CDB7DEB72D970FB6F894DEBF0FBECDBF71
:101B50000E947911282E81110E94490D83E292E0A2
:101B60009D878C8700E010E0302E802F0E9484102B
:101B70002B013C01EC85FD8581919191A191B19161
:101B8000FD87EC875301420188269926AA26BB26A9
:101B900081149104A104B104B1F40F5F1F4F06300A
:101BA000110511F78FEF89838A831B820E9490159C
:101BB0008160782F9D838C8349815A816B818D81CF
:101BC0000E94E00251C08091430281FD0E9490106A
:101BD0001B86C12CD12C7601C394D501C4018C2164
:101BE0009D21AE21BF21892B8A2B8B2B91F10E9445
:101BF000650D8823D1F0FB85FE833F824C205D205C
:101C00006E207F2081E045284628472809F480E09F
:101C100088870E9490158160782F9A8789874E81E6
:101C20005F8168858A850E94E002000F111F000F06
:101C3000111FF801ED5DFD4F80819181A281B3817B
:101C4000C826D926EA26FB26C082D182E282F38208
:101C50000BC08B858F5F8B87CC0CDD1CEE1CFF1CB3
:101C6000813109F0BACF99CF81E0211001C080E025
:101C70002D960FB6F894DEBF0FBECDBFDF91CF918A
:101C80001F910F91FF90EF90DF90CF90BF90AF909A
:101C90009F908F907F906F905F904F903F902F908C
:101CA00008950E948E0D0C94D502CF93DF930E946D
:101CB0006F0FEC01811522E59207E8F5811531E5FA
:101CC000930708F0B6C0883E910528F5803E91053F
:101CD00008F0E9C0883A910570F4853A910508F05A
:101CE0007AC08130910509F473C008F4D9C0049713
:101CF00008F0D9C0D5C08F3B910508F0D1C0C85AB3
:101D0000D0E0CC0FDD1FCE5BDE4F0990D881C02D17
:101D1000CE019464C9C0811540E5940708F069C0FC
:101D2000811550E4950708F060C09A9581159F4190
:101D300008F4B9C0B5C0811536E5930728F58115BB
:101D400045E5940708F092C0811554E5950708F021
:101D500087C0AC0143705527282F26952695C115BD
:101D6000D34508F06CC081E090E002C0880F991F55
:101D70004A95E2F740E2249F90011124EC01C22B26
:101D8000D32BCE019C6890C081152AE5920780F480
:101D9000811539E5930708F072C0811548E594076D
:101DA00008F47EC0D82FCC27CE01806F906A7CC00B
:101DB00090568115904208F073C08D2F8F710E944C
:101DC0000310DD27D0628F71AE01582BCA016CC0A1
:101DD00081E090E069C0C55AD0E0C059DE4F8881EB
:101DE000C82FD0E0CE0190645FC0DF70CE01906A52
:101DF0005BC074E0969587957A95E1F7282F23705C
:101E00003C2F337081E090E002C0880F991F3A9513
:101E1000E2F79C68AC01522B9A019C2F9F7096951B
:101E2000969550E2959FE0011124C9018C2B9D2BC2
:101E30003BC0D82FCC27CE01816F906A35C081E09E
:101E400090E002C0880F991F4A95E2F750E2259F63
:101E500090011124EC01C22BD32BCE019A6824C02F
:101E6000D82FCC27CE01846F906A1EC00E94031029
:101E70008F7190E0D82FCC27CE01906215C08F7063
:101E80000E94031094E0D695C7959A95E1F7CF701C
:101E9000D0E0DC2FCC27D0699E01282BC90104C0DB
:101EA00080E090E001C0CE01DF91CF91089526E659
:101EB000829FC0011124FC0121E1729FE00DF11D00
:101EC0001124E60FF11DEE0FFF1FE852FF4F859121
:101ED000949108950E94570F0E94550E08958238DC
:101EE000910569F1B0F48133910509F46DC048F4AE
:101EF0008932910509F463C08A32910509F469C0F9
:101F000008958533910509F455C089339105B9F0D9
:101F10000895833E910569F138F4803E9105B1F052
:101F2000823E910509F10895863E9105A9F1873E0B
:101F30009105B9F1843E910509F064C023C0209158
:101F4000600220FD4FC021FD4DC0089580916002C8
:101F500080FD44C08091610280FF44C08091600296
:101F600084FD42C083EE4DC08091600282FF38C084
:101F7000F5CF8091600282FD33C08091610280FDC7
:101F800031C0ECCF8091610281FF32C0809160024C
:101F900084FD2AC087EE35C08091600283FF26C091
:101FA000F5CF8091600283FD21C08091610281FDA7
:101FB0001FC0ECCF8091600285FD1CC01DC08091C8
:101FC000600285FD19C016C08091600286FD16C0B2
:101FD00017C08091600286FD13C010C089E311C054
:101FE00082EE0FC080EE0DC080E00BC086EE09C00F
:101FF00084EE07C089E205C085E303C08AE201C020
:1020000081E390E008959091600292FF0DC0282F27
:102010002871283019F4877F846006C0282F247126
:10202000243011F48B7F886093FF0DC0282F287116
:10203000283119F4877E846106C0282F2471243149
:1020400011F48B7E88612091610220FF0DC0382F32
:102050003871383019F4877F816006C0382F3171AC
:10206000313011F48E7F886021FF0DC0282F287138
:10207000283119F4877E816106C0282F2171213112
:1020800011F48E7E886194FD877E089580E0089526
:102090000C94940C0E9479118FE39CE90197F1F75D
:1020A00000C000000E94791180E00E94841060FF4F
:1020B00004C00E9448100C94DD1508950C944A1039
:1020C0000E949A0C811102C00E94420D0E94A50C30
:1020D000809343020E94AD0C909361028093600252
:1020E0000E945E100E94A90C682F70E080E090E0D2
:1020F0000E94B6066091CF017091D0018091D1010C
:102100009091D2010C94EE0624E0829FC00111242C
:10211000FC01E658FD4F60817181828193810895B1
:10212000089580EA8A95F1F7089500C008950C9407
:10213000911008950C9499100C949A100C94991085
:102140000C949E10F894E82FE295EF70F0E031A126
:10215000282F2F7081E090E001C0880F2A95EAF7C0
:10216000982F9095932391A392A1892B82A3789481
:1021700008950F931F93CF93DF93C4E8D1E0899123
:102180008F3F11F00E94A21081E0CA38D807B9F73A
:10219000C3E7D1E004E811E089918F3F11F00E947C
:1021A000A2100C171D07C1F7DF91CF911F910F915E
:1021B00008954F925F926F927F928F929F92AF920B
:1021C000BF92DF92EF92FF920F931F93CF93DF9313
:1021D0008C01C62FD0E0CE018C579E4F7C01FC01B4
:1021E00090819F3F09F460C0D62EF894E92FE295C4
:1021F000EF70F0E081A19F7021E030E001C0220F7C
:102200009A95EAF7822B81A382A12095282322A305
:1022100078940E949510E3E7F1E024E831E0412C46
:10222000512C32014394812C912C540181918F3F88
:1022300099F0A82FA295AF70B0E090964C9150E025
:102240008F70BA0102C0759567958A95E2F760FDB7
:1022500003C0D301C20103C080E090E0DC01882A02
:10226000992AAA2ABB2A440C551C661C771C2E17D7
:102270003F07E1F6F70180818F3F11F00E94A21025
:1022800061E081149104A104B10409F460E08D2D92
:102290000E949710CC0FDD1FCC0FDD1FC00FD11F88
:1022A00088829982AA82BB82DF91CF911F910F9180
:1022B000FF90EF90DF90BF90AF909F908F907F90B6
:1022C0006F905F904F9008950E94B91088E1EAE7FF
:1022D000F2E0DF01982F1D929A95E9F7E2E6F2E02D
:1022E000DF011D928A95E9F786E00E94C4110C94E3
:1022F0003A02FF920F931F93CF93DF93CDB7DEB7D0
:1023000068970FB6F894DEBF0FBECDBF8E010F5F8A
:102310001F4F88E1F80111928A95E9F7F12C6F2D92
:10232000C8010E94D910F394F6E0FF12F8CF48E1FB
:1023300050E0B80182E692E00E94B51CFF24F394BD
:10234000009709F4F12C892B41F088E1F801A2E60D
:10235000B2E001900D928A95E1F72F2D46E06AE7F1
:1023600072E082E692E00E94C5110E943C028F2D2D
:1023700068960FB6F894DEBF0FBECDBFDF91CF9148
:102380001F910F91FF9008950895FF920F931F934F
:10239000CF93DF93F82ED92F8B01C42F222349F03E
:1023A00081E0809346020E949015909345028093AD
:1023B0004402809146028823F1F08091440290917A
:1023C00045020E94A8150597B0F0EF2DFD2FD8010A
:1023D00080E090E04C2F50E08417950754F4019171
:1023E0001191219131910D931D932D933D93019660
:1023F000F3CF10924602DF91CF911F910F91FF9082
:1024000008950E9475170E94860D0C9481170E94F2
:1024100085170E94510E0C949F170E942E150E9442
:102420005C170E94740D0E9401120E9407120E9404
:102430007E0DFBCFCF93DF93EC01FB0182818823DC
:1024400009F43CC1C430FDE5DF0760F4CB3F9CE5F7
:10245000D90788F49E0122503C452431310508F00B
:102460002EC109C0C236EDE5DE0729F0C63AFDE50A
:10247000DF0709F024C10E94AD0C909361028093A4
:102480006002C1318CE5D80709F4C6C008F042C02B
:10249000C930ECE5DE0709F49BC000F5C5308CE5DA
:1024A000D80709F485C078F4C330ECE5DE0709F4F9
:1024B00078C008F07AC0C230DC4509F0F5C08091E0
:1024C00060028160EFC0C7309CE5D90709F478C08D
:1024D00008F07AC0809160028061E4C0CD30FCE5F4
:1024E000DF0709F487C058F4CB309CE5D90709F41D
:1024F00079C008F07BC08091600288606FC0CF30E7
:10250000FCE5DF0709F480C008F082C0809160021A
:10251000877FC8C0CE3F9CE5D90709F471C000F59C
:10252000C531FCE5DF0709F485C068F4C3319CE5DB
:10253000D90709F475C008F095C00E945E06809125
:1025400060028F77AFC0CC3FFCE5DF07A9F108F050
:1025500054C0CB3FDC4509F0A7C08091610240C068
:10256000C230EDE5DE0709F489C058F4C1158DE5E8
:10257000D80709F45AC008F069C0809161028260EE
:102580002FC0C236EDE5DE0709F47CC0C63AFDE592
:10259000DF0709F481C0C330DD4509F085C080E064
:1025A0006EC08091600282607DC08091600216C022
:1025B00080916002886076C08091610282604FC025
:1025C0008091600280626EC08091600280646AC007
:1025D0000E945E0680916002806864C0846062C070
:1025E00081603DC0809160028E7F5CC080916002FE
:1025F0008D7F58C08091600216C08091610218C022
:10260000809161028D7F2BC0809160028F7E4AC0D5
:10261000809160028F7D46C0809160028F7B42C0B6
:1026200080916002877F8B7F3DC0809161028D7FAA
:102630008E7F15C08091600282FB222720F991E0F5
:10264000922790FB82F990FB83F92CC08091610264
:10265000982F909591708E7F892B90FB81F98093B4
:10266000610222C00E945E068091600287FB2227E1
:1026700020F991E0922790FB87F914C081E00E9435
:10268000440D12C08091600284FB222720F991E062
:10269000922790FB84F906C080916002982F909554
:1026A00090FB80F9809360028091600290916102BA
:1026B0000E94BE0C0E945E0680E001C081E0DF91B6
:1026C000CF910895CF93DF9386319C4541F5EB017F
:1026D0000E94B10B982F8A81209102013091030151
:1026E000882379F09A7A81E009F480E080934702A8
:1026F000911102C069E201C065E3C9010E94E714BB
:102700000AC080914702811102C069E201C065E3FD
:10271000C9010E94E9140E94F30B80E001C081E02E
:10272000DF91CF9108950F931F93CF93DF93C42F21
:10273000D22FFC0182818823C9F040934A020E9473
:102740009015909349028093480280E28C0F883064
:1027500008F057C0C77081E001C0880FCA95EAF73A
:10276000DF91CF911F910F910C94CA0380914A027F
:10277000481330C080914802909149020E94A815E8
:10278000883C910538F510E21D0FCD17B9F080E2B5
:102790008C0F883040F4C77081E001C0880FCA9563
:1027A000EAF70E94D103183028F581E09D2F977039
:1027B00001C0880F9A95EAF70E94CA03802F0E94F1
:1027C000C1031830F0F4D77081E001C0880FDA95AA
:1027D000EAF70AC080E28C0F883098F4C77081E075
:1027E00001C0880FCA95EAF7DF91CF911F910F9131
:1027F0000C94D103802FDF91CF911F910F910C94F6
:10280000C103DF91CF911F910F9108950F939C0108
:10281000CB01243F4CE5340731F188F4293DFCE538
:102820003F07D9F02A3D4CE5340779F1283D3C4576
:10283000A9F506E221EE41EE68ED7CE52BC0263FCE
:10284000FCE53F07E1F0A8F0273F3C4539F507E2FA
:1028500025EE46EE67EF7CE51DC007E225EE45EE6E
:1028600069ED7CE517C006E221EE40EE64EF7CE501
:1028700011C007E225EE44EE65EF7CE50BC006E2F1
:1028800021EE42EE66EF7CE505C008E221E045EE70
:102890006AED7CE50E94931380E008C0FC01828110
:1028A000882319F010924A0201C081E00F91089527
:1028B00090938B0180938A010895909350028093A6
:1028C0004F020895E0914F02F0915002309721F0AD
:1028D0000190F081E02D099480E00895E0914F028D
:1028E000F0915002309721F00280F381E02D09949D
:1028F000089520914D0230914E022817390771F04A
:1029000090934E0280934D02E0914F02F09150025D
:10291000309721F00680F781E02D099408952091E9
:102920004B0230914C022817390771F090934C02FA
:1029300080934B02E0914F02F0915002309721F0CA
:102940000084F185E02D09940895FC01329697E00A
:1029500080E0915029F021912223D9F38F5FF9CFA4
:102960000895662349F0FC0132960896219162177A
:1029700029F0E817F907D1F780E0089581E008957C
:102980009C01FC0132969FEF80E04191461789F04F
:102990009F3F19F4411101C0982F8F5F8630A9F72E
:1029A0009F3F39F0F901E90FF11D97FDFA95628318
:1029B000089508959C012A5F3F4FFC014281461310
:1029C00001C01282019682179307B9F708950C94FB
:1029D000C0140C94DA14029626E0FC0111922A9598
:1029E000E9F7089508950C94F21483E0809351025E
:1029F0000C94F314811102C081E001C082E0809345
:102A000051020C94F3140C94FA1481E08093510257
:102A10000C94F3140C94051508950C940C150C9457
:102A20000D150C940C150C940C150C940C15CF93DF
:102A30000E9413150E9479110E941115C0E08C2F7D
:102A40000E948410672B682B692B29F4CF5FC63056
:102A5000B1F780E001C081E0CF91089508951F9201
:102A60000F920FB60F9211248F939F93AF93BF9342
:102A700080915202811113C0809192029091930231
:102A8000A0919402B09195024196A11DB11D809331
:102A9000920290939302A0939402B0939502BF91F7
:102AA000AF919F918F910F900FBE0F901F9018952F
:102AB00080919A02843031F10E94A0021092520259
:102AC00020E488E190E00FB6F894A8958093600028
:102AD0000FBE2093600083B7817F846083BF83B77C
:102AE000816083BF7894889583B78E7F83BF0FB64C
:102AF000F894A8958091600088618093600010929E
:102B000060000FBE08950E945E060C94A40282E04D
:102B100084BD93E095BD9AEF97BD80936E000895B4
:102B20002FB7F8948091920290919302A091940211
:102B3000B09195022FBF08952FB7F894609192023B
:102B40007091930280919402909195022FBF089505
:102B50009C014FB7F8948091920290919302A091BA
:102B60009402B09195024FBF821B930B0895789405
:102B70001F920F920FB60F9211248F939F93AF93D2
:102B8000BF938091920290919302A0919402B09190
:102B900095020196A11DB11D80939202909393021C
:102BA000A0939402B0939502BF91AF919F918F91A2
:102BB0000F900FBE0F901F90189581E08093E0005A
:102BC00080E28093D8001092C9008FE19EE40197C3
:102BD000F1F700C0000087E090EBDC018093A302D6
:102BE0009093A402A093A502B093A6029CE088E172
:102BF0000FB6F894A895809360000FBE9093600084
:102C0000FFCF80915E0208950895CF93DF9321E076
:102C10002093E9002FEF3091E800215035FD06C0E8
:102C200035ED3A95F1F700002111F5CF2091E8003C
:102C300025FF14C0EC0140E050E068E070E00E9425
:102C400011188091E8008E778093E80088E0FE01FB
:102C5000A6E5B2E001900D928A95E1F7DF91CF9160
:102C600008958093530270935502609354028091AB
:102C70009A02843001F582E08093E9008FEF909111
:102C8000E800815095FD06C095ED9A95F1F700009A
:102C90008111F5CF8091E80085FF0DC040E050E044
:102CA00063E070E083E592E00E9411188091E800F3
:102CB0008E778093E8000895BC0184E00C9431166F
:102CC000BC0183E00C943116089580919902811122
:102CD00009C00E94A2190E94FF198091E20084603D
:102CE0008093E20008951092990208950C940A15B9
:102CF0006091960281E0611101C080E00C94F514AE
:102D000090919A0281E0943009F080E060919602FF
:102D10000C94FA1442E061EC81E00E941B1942E23B
:102D200061EC82E00E941B1990919A0281E094303C
:102D300009F080E0609196020C94031580919C024A
:102D4000833009F461C030F4813071F0823009F4CD
:102D50009AC008958A3009F486C08B3009F46CC09B
:102D6000893009F0A8C020C080919B02813A09F007
:102D7000A2C08091E800877F8093E80080919F0245
:102D80009091A002892B21F468E086E592E003C0CF
:102D900060E080E090E070E00E945C188091E800C4
:102DA0008B778093E800089580919B02813209F02F
:102DB00082C080919F029091A002029708F07BC090
:102DC0008091E800877F8093E8008091E80082FD91
:102DD00005C080919A028111F8CF6DC02091F30057
:102DE0008091F20090E0922B029731F48091F100F3
:102DF000813011F0863021F48091F10080935E02E1
:102E00008091E8008B7753C080919B02813A09F052
:102E100052C080919F029091A002892B09F04BC073
:102E20008091E800877F8093E8008091E80080FF30
:102E3000FCCF8091100136C080919B028132D9F580
:102E400080919F029091A002892BA9F58091E800C2
:102E5000877F8093E8000E94501980919D028093A3
:102E600010010C945E0680919B02813221F58091C5
:102E7000E800877F8093E8000E94501980919E02AD
:102E800080935F02089580919B02813AA1F4809122
:102E9000E800877F8093E8008091E80080FFFCCF06
:102EA00080915F028093F1008091E8008E7780939B
:102EB000E8000C945019089584B7877F84BF0FB63B
:102EC000F894A895809160008861809360001092CA
:102ED00060000FBE90E080E80FB6F8948093610028
:102EE000909361000FBE0C9405150E94A2190E94D8
:102EF000FF19E2EEF0E080818460808378940C9486
:102F0000941C84E091E00C945D1480919A028530C9
:102F1000A9F480919A02853079F40E945815809125
:102F200098028823B1F30E941715882391F30E9419
:102F3000FB170E945E06EDCF0C948315089508954B
:102F40000C94A217292F332723303105C9F060F4E0
:102F50002130310581F02230310509F044C08BE386
:102F600090E02CE932E043C021323105E1F0223219
:102F7000310549F138C082E190E027ED32E037C0F9
:102F800099278130910549F028F0029761F5E0E733
:102F9000F2E005C0E8E9F2E002C0E2E8F2E0849184
:102FA00090E09F0124C06115710541F06130710509
:102FB000D1F489E090E027EC32E019C089E090E09C
:102FC0002EEA32E014C06115710541F061307105DF
:102FD00051F482E390E029EE32E009C080E490E011
:102FE0002BE133E004C080E090E020E030E0FA0123
:102FF00031832083089580E189BD82E189BD09B4D0
:1030000000FEFDCF8091D8008F7D8093D800809105
:10301000E00082608093E0008091E00081FDFCCFC1
:103020000895CF92DF92EF92FF920F931F93CF9369
:10303000DF93EC018B017A010E946F19811133C07B
:10304000E114F10439F0F70180819181081B190B1B
:10305000C80FD91FC12CD12C0115110519F1809170
:10306000E80085FD16C08091E8008E778093E80027
:10307000E114F10449F0F70180819181C80ED91E55
:10308000D182C08285E00FC00E946F19882321F38E
:103090000AC089918093F10001501109FFEFCF1A06
:1030A000DF0ADACF80E0DF91CF911F910F91FF907F
:1030B000EF90DF90CF9008952091A1023091A2026D
:1030C0002617370748F06115710539F42091E8009B
:1030D0002E772093E80001C0B901FC0120E06115C2
:1030E000710579F180919A028823F1F18530F1F12F
:1030F0008091E80083FD3CC08091E80082FD2EC0F5
:103100008091E80080FFEBCF2091F3008091F200E6
:1031100090E0922B6115710551F08830910538F4DB
:1031200021912093F100615071090196F3CF21E0C4
:10313000089709F020E08091E8008E778093E800FE
:10314000CECF2111CFCF0AC080919A02882361F09F
:10315000853061F08091E80083FD0AC08091E8002D
:1031600082FFF2CF80E0089582E0089583E0089521
:1031700081E008952091A1023091A202261737071D
:1031800048F06115710539F42091E8002E772093FD
:10319000E80001C0B901FC0120E06115710591F161
:1031A00080919A02882309F440C0853009F43FC019
:1031B0008091E80083FD3DC08091E80082FD2FC032
:1031C0008091E80080FFE9CF2091F3008091F20028
:1031D00090E0922B6115710559F08830910540F40B
:1031E00024912093F1003196615071090196F2CF3C
:1031F00021E0089709F020E08091E8008E77809325
:10320000E800CBCF2111CCCF0AC080919A0288234D
:1032100061F0853061F08091E80083FD0AC0809103
:10322000E80082FFF2CF80E0089582E0089583E015
:10323000089581E00895982F973068F59093E900FC
:10324000981739F07091EC002091ED005091F0004A
:1032500003C0242F762F50E021FD02C09F5FECCFEA
:103260003091EB003E7F3093EB003091ED003D7FDD
:103270003093ED003091EB0031603093EB007093B0
:10328000EC002093ED005093F0002091EE0027FD1C
:10329000E5CF80E008958F708093E90081E0089584
:1032A00080919B0287FF11C08091E80082FD05C0DC
:1032B00080919A028111F8CF11C08091E8008B773C
:1032C0000BC080919A02882349F08091E80080FF2A
:1032D000F8CF8091E8008E778093E80008952091E0
:1032E000E4003091E50095E64091EC00842F817078
:1032F00040FF23C08091E80080FD1DC080919A02AC
:10330000882399F0853099F08091EB0085FD11C0FC
:103310004091E4005091E5002417350729F39150BE
:1033200011F09A01E1CF84E0089582E0089583E0EE
:10333000089581E0089580E008954091E80042FFFB
:10334000DDCF08950E94101A0E94181AE0EEF0E0F6
:10335000808181608083E8EDF0E080818F778083D9
:1033600019BCA7EDB0E08C918E7F8C9380818F7E0D
:1033700080831092990208950F931F93CF93DF9348
:103380000E94101A0E94181AC8EDD0E088818F7729
:10339000888388818068888388818F7D888319BC31
:1033A00010929A021092960210929802109297022E
:1033B00000EE10E0F80180818B7F8083888181603E
:1033C000888342E060E080E00E941B19E1EEF0E0BB
:1033D00080818E7F8083E2EEF0E080818160808357
:1033E000808188608083F80180818E7F80838881DE
:1033F00080618883DF91CF911F910F910895E8ED4F
:10340000F0E080818F7E8083E7EDF0E08081816055
:10341000808384E082BF81E0809399020C94BC1980
:10342000E8EDF0E080818E7F80831092E2000895C5
:103430001092DA001092E10008951F920F920FB6D9
:103440000F9211242F933F934F935F936F937F932A
:103450008F939F93AF93BF93EF93FF938091E1007E
:1034600082FF0BC08091E20082FF07C08091E100E3
:103470008B7F8093E1000E94931C8091DA0080FF93
:103480001FC08091D80080FF1BC08091DA008E7F22
:103490008093DA008091D90080FF0DC080E189BD62
:1034A00082E189BD09B400FEFDCF81E080939A02DC
:1034B0000E94651605C019BC10929A020E947316EC
:1034C0008091E10080FF19C08091E20080FF15C06B
:1034D0008091E2008E7F8093E2008091E200806123
:1034E0008093E2008091D80080628093D80019BC5C
:1034F00085E080939A020E9478168091E10084FF13
:1035000030C08091E20084FF2CC080E189BD82E15F
:1035100089BD09B400FEFDCF8091D8008F7D8093D6
:10352000D8008091E1008F7E8093E1008091E200DD
:103530008F7E8093E2008091E20081608093E200C0
:1035400080919602882311F084E007C08091E30007
:1035500087FD02C081E001C083E080939A020E944F
:1035600080168091E10083FF29C08091E20083FFF3
:1035700025C08091E100877F8093E10082E0809305
:103580009A02109296028091E1008E7F8093E10072
:103590008091E2008E7F8093E2008091E200806162
:1035A0008093E20042E060E080E00E941B1980917D
:1035B000F00088608093F0000E947616FF91EF91F2
:1035C000BF91AF919F918F917F916F915F914F913B
:1035D0003F912F910F900FBE0F901F9018951F9243
:1035E0000F920FB60F9211242F933F934F935F9337
:1035F0006F937F938F939F93AF93BF93CF93DF93FB
:10360000EF93FF93C091E900CF708091EC00D82F29
:10361000D17080FDD0E81092E9008091F000877FA2
:103620008093F00078940E94331B1092E9008091FF
:10363000F00088608093F000CD2BCF70C093E9003C
:10364000FF91EF91DF91CF91BF91AF919F918F91BA
:103650007F916F915F914F913F912F910F900FBE8E
:103660000F901F9018951F93CF93DF93CDB7DEB7C0
:10367000AA970FB6F894DEBF0FBECDBFEBE9F2E01C
:103680008091F100819322E0E33AF207C9F70E94AA
:103690009E168091E80083FF2EC180919B0290913D
:1036A0009C02492F50E04A30510508F024C1FA012C
:1036B000EE59FF4F0C94AF1C803821F0823809F08E
:1036C0001AC108C08091970290919802992389F0BD
:1036D00082600FC080919F028F70873008F00BC10D
:1036E0008093E9008091EB0085FB882780F9109298
:1036F000E9009091E800977F9093E8008093F100B3
:103700001092F100D1C0282F2D7F09F0F4C088233A
:1037100019F0823061F0EFC080919D02813009F094
:10372000EAC0933009F080E0809398022EC0809127
:103730009D0281112AC080919F028F702FEF280F68
:10374000263008F0D8C08093E9002091EB0020FFDC
:103750001CC0933021F48091EB00806214C09091E2
:10376000EB0090619093EB0021E030E0A90102C0F2
:10377000440F551F8A95E2F74093EA001092EA0041
:103780008091EB0088608093EB001092E9008091BB
:10379000E800877F8093E8000E945019ACC0811137
:1037A000AAC010919D021F778091E3008078812B41
:1037B0008093E3008091E800877F8093E8000E9477
:1037C00050198091E80080FFFCCF8091E300806871
:1037D0008093E300111102C082E001C083E0809376
:1037E0009A0289C08058823008F085C080919D027D
:1037F00090919E028C3D53E0950779F583E08A8392
:103800008AE289834FB7F894DE01139620E03EE008
:1038100051E2E32FF0E050935700E49120FF03C002
:10382000E295EF703F5FEF708E2F90E0EA3010F07E
:10383000C79601C0C0968D939D932F5F243149F7A1
:103840004FBF8091E800877F8093E8006AE270E0D4
:10385000CE0101960E945C1816C060919F02709183
:10386000A002AE014F5F5F4F0E94A017BC01892BE1
:1038700009F441C09091E800977F9093E800898116
:103880009A810E94BA188091E8008B778093E800B3
:1038900032C0803881F58091E800877F8093E8000E
:1038A000809196028093F1008091E8008E7772CF2C
:1038B000811121C080919D0290919E0299270297CB
:1038C000D4F48091E800877F8093E80080919D0286
:1038D000809396020E94501980919602811106C031
:1038E0008091E30087FD02C081E001C084E0809305
:1038F0009A020E948A168091E80083FF0AC0809194
:10390000E800877F8093E8008091EB0080628093DD
:10391000EB00AA960FB6F894DEBF0FBECDBFDF91C5
:10392000CF911F9108950895CF9380919A02882393
:10393000A1F0C091E900CF709091EC00892F8170C7
:1039400090FD80E8C82B1092E9008091E80083FD8B
:103950000E94331BCF70C093E900CF910895EE0F02
:10396000FF1F0590F491E02D0994FB01DC0104C0D8
:103970008D910190801921F441505040C8F7881B67
:10398000990B0895F999FECF92BD81BDF89A9927B8
:1039900080B50895A8E1B0E042E050E00C94F61C38
:1039A000262FF999FECF92BD81BDF89A019700B4F8
:1039B000021639F01FBA20BD0FB6F894FA9AF99A98
:1039C0000FBE08950396272F0E94D11C0E94D01C81
:1039D000252F0E94D11C242F0C94D11C0196272F37
:1039E0000E94D11C0C94D01CDC01CB01FC01F99984
:1039F000FECF06C0F2BDE1BDF89A319600B40D923B
:0C3A000041505040B8F70895F894FFCFF3
:103A0C00C800190201160516641660165C16041619
:103A1C0001E200E900EA00B500B600B700CD008372
:103A2C0001CC008A01920194012102230224022577
:103A3C0002260227022A02B300B4006F0070008134
:103A4C008283E200E900EA00B500B600B700CD00C1
:103A5C008301CC008A0192019401210223022402E9
:103A6C002502260227022A02B300B4006F00700060
:103A7C00818283F0F1F4F5F6F76766363534979466
:0A3A8C0096929395919033303231F9
:00000001FF
